:020000040800F2
:1000000000040220010200080302000803020008A5
:1000100003020008030200080302000803020008AC
:1000200003020008030200080302000889260008F2
:10003000030200080302000803020008030200088C
:10004000030200080302000803020008030200087C
:1000500003020008030200089D380008C9380008A0
:10006000F5380008213900084D390008030200085E
:10007000030200080302000803020008030200084C
:10008000030200080302000803020008030200083C
:10009000030200080302000803020008793900087F
:1000A000030200080302000803020008030200081C
:1000B000C13600080302000803020008030200081A
:1000C00003020008030200080302000803020008FC
:1000D00003020008030200080302000803020008EC
:1000E000E1390008030200080302000803020008C7
:1000F00003020008030200080302000803020008CC
:1001000003020008030200080302000803020008BB
:1001100003020008030200080302000803020008AB
:10012000030200080302000803020008030200089B
:10013000030200080302000803020008030200088B
:10014000030200080302000803020008F12D000862
:10015000030200080302000803020008030200086B
:10016000030200080302000803020008030200085B
:10017000030200080302000803020008030200084B
:100180000302000803020008910F000803020008A0
:10019000030200080302000803020008030200082B
:1001A000030200080302000803020008030200081B
:1001B000030200080302000803020008030200080B
:1001C00003020008030200080302000803020008FB
:1001D00003020008030200080302000803020008EB
:1001E00003020008030200080302000803020008DB
:1001F00003020008030200080302000803020008CB
:1002000002E000F000F8FEE772B6384880F3088894
:10021000374880F3098837484EF60851CEF200017E
:10022000086040F20000CCF200004EF63471CEF2CD
:1002300000010860BFF34F8FBFF36F8F40F20000E3
:10024000C0F2F0004EF68851CEF200010860BFF314
:100250004F8FBFF36F8F4FF00000E1EE100A4EF6A4
:100260003C71CEF200010860062080F31488BFF3D1
:100270006F8F02F047FA03F0ABF91F481F491B4A82
:1002800091423CBF41F8040BFAE71D49184A9142DC
:100290003CBF41F8040BFAE71A491B4A1B4B9A4230
:1002A0003EBF51F8040B42F8040BF8E70020184950
:1002B000184A91423CBF41F8040BFAE702F060FA99
:1002C00003F0F0F9144C154DAC4203DA54F8041B5A
:1002D0008847F9E700F040F8114C124DAC4203DAC0
:1002E00054F8041B8847F9E702F048BA00040220DA
:1002F000002402200000000855555555000002203A
:1003000000040220603E0008002402204C24022049
:1003100050240220E03802200002000800020008F9
:1003200000020008000200082DE9F04F2DED108AB0
:10033000C1F80CD0D0F80CD0BDEC108ABDE8F08F1D
:10034000002383F311882846A047002001F026FEF1
:1003500001F0D6FD00DFFEE770B5214C6FF07203AF
:10036000002523706FF07F061E236570A570E57071
:1003700025716571A571E57125726672A372E572CA
:1003800000F014FD20B10E2325726672A372E5728F
:1003900002F052F9044602F071F960B9114B9C4227
:1003A0000CD001339C4218BF002541F2883404BFB1
:1003B0000125002404E00024012501E0044605464F
:1003C000002002F043F90DB100F0B2F800F070FD2A
:1003D00000F040FC204600F041F900F0A9F8F9E7F0
:1003E00050240220010007B008B500F0BDFBA0F1C9
:1003F00020035842584108BD07B5054B01A81B888A
:10040000ADF80430022100F00FFC03B05DF804FBEE
:10041000E03A0008064991F8243033B10023086A15
:1004200081F82430082200F037BC0120704700BF5B
:10043000702902202DE9F047224C94F8243005461B
:10044000884617460BB92E4631E0266A06EB83062E
:10045000B0422CD0FFF7DEFF0028F4D10020BDE829
:10046000F08794F824901748B9F1000F04D1FF21C8
:100470002022066200F00AFDC9F10805BD4228BF2E
:100480003D465FFA85FAAD00414604EB89002A46F5
:1004900000F0D2FC94F824305344DBB2CAEB0707D7
:1004A000082B2E44A844FFB284F8243002D0002F39
:1004B000D7D104E0FFF7AEFF0028F8D1CEE7012046
:1004C000BDE8F0877029022008B5202383F3118846
:1004D0001348C3680BB101F0E7FD1148114A4FF40E
:1004E0007A71002301F0A4FD002383F311880E4BE1
:1004F0001A6812B11A68013A1A605A680A4912B1A8
:100500004A68013A4A60094A12783AB95B682BB9DD
:10051000022000F07FFC044B32225A6008BD00BF6D
:100520005C240220C90400089C290220982902208A
:10053000F8B5404B53F8042F01327AD03E4A93422B
:10054000F8D13E4C3E4B22689A4272D93D4B9B6893
:1005500003F1006303F5C0339A426AD2002000F031
:1005600093FB394B0220187000F046FC374B1A6C95
:1005700000221A64196E1A66196E596C5A64596E03
:100580005A66596E596941F080015961596921F0E3
:10059000800159615969196941F00051196119695E
:1005A00021F0005119611B6972B62949294B0B6072
:1005B0001D682668BFF34F8FBFF36F8F264BC3F8BC
:1005C0008420BFF34F8F5A6922F480325A61BFF3FF
:1005D0004F8FD3F88030C3F34E32C3F3C9015301B8
:1005E00043F6E0741C4008461B4B44EA807710F148
:1005F000FF30C3F87472F7D212F1FF32EFD2BFF3BB
:100600004F8FBFF36F8FBFF34F8FBFF36F8F5A6959
:1006100022F400325A610022C3F85022BFF34F8FF8
:10062000BFF36F8F202383F31188AD4685F30888CD
:100630003047F8BDFC7F01081C80010804800108D8
:10064000FF7F010850240220982902200038024030
:1006500008ED00E00080010800ED00E02DE9F04F1A
:10066000B74F97B020228146FF210EA8BC6800F04A
:100670000DFCB44A1378A3B9B3480121C3601170CB
:10068000202383F31188C3680BB101F00DFDAE4840
:10069000AE4A4FF47A71002301F0CAFC002383F3C1
:1006A0001188DFF8BCA2B9F1000F01D0CAF80090A0
:1006B000A74B00251D70CAF8045000952E46984699
:1006C000012000F099FBB9F1000F04D0DAF80030F6
:1006D000002B00F03C82002000F046FA0290029BC2
:1006E000002BF0DB012000F079FB029B213B122B59
:1006F000E6D801A252F823F0450700085707000882
:10070000C5070008C1060008C1060008C1060008A8
:1007100047080008690A000801090008C70900081D
:10072000FD0900082B0A0008C1060008430A00085A
:10073000C1060008B10A0008210B0008C106000824
:10074000ED0A00080220FFF74FFE002800F0F481B8
:1007500001230093E4E14FF47A7000F005FAB0F160
:10076000000BC0F2E9810220FFF73EFE002800F0F6
:10077000E3810BF1FF30042800F2DD81DFE800F0B7
:1007800003080A0F110016A8052340F8343D02E0C3
:100790006B4800E06F48042100F046FA0FE06E4815
:1007A000F9E71C25284600F071FA16AB042143F83E
:1007B000340D0435184600F037FA2C2DF2D10125FE
:1007C0000026ADE1009B002B00F0B681002D00F06B
:1007D000B3810220FFF708FE002800F0AD81012060
:1007E00000F052FA022088F8000000F005FB4FF0FC
:1007F000000B5FFA8BF21046019200F055FA019A55
:1008000038B1104600F060FA0BF1010B0028F0D16E
:1008100094E101900122022088F8002000F0DEFA25
:10082000019B1C46BB689C4207D2204600F02EFA72
:10083000013040F083810434F4E7002488F800405C
:10084000CAF804406CE1009B002B00F07581002D7C
:1008500000F07281022088F8000000F0CDFA32200A
:1008600000F082F9B0F1000BC0F266811BF00303C7
:1008700040F06281B9680BEB04028A4200F25C81AD
:10088000BBF5807F00F258815B450FDA4FF47A7038
:10089000019300F069F90290029A002AC0F24C819B
:1008A000019B2E4A029999540133EDE7C820FFF7C6
:1008B0009BFD002800F040811F2C13D8C4F12003B9
:1008C0005B4528BF5B460EAA24F003001044234971
:1008D00001931A4600F0B0FA019B2048FF211A4606
:1008E00000F0D4FA4FEAAB0B20461C495FFA8BF2BA
:1008F000FFF7A0FD002800F0218104EB8B040FE13D
:100900000220FFF771FD002800F01681FFF782FD3D
:10091000002800F011814FF0000B5946BB689B4541
:100920004DD2BBF1200F1DD20E9B01331AD02BF0FC
:10093000030316AA134453F8203C099318E000BFA0
:1009400050240220A42902205C240220C9040008AB
:1009500098290220542402205824022070240220C6
:100960009C2902205846019100F090F901990990C4
:10097000784B5B689BB91A46082012F0010F4FEACA
:10098000520E16BF744A72468EEA02020138F4D142
:10099000704840F823200133B3F5807FEBD100226B
:1009A00009AB6C48D35C4B40DBB2013250F82330CA
:1009B000042A83EA1121F3D10BF1040BAEE716A848
:1009C00040F84C1D16E016A8002340F8343D642181
:1009D00000F0FCF8002840F0AF800220FFF704FD93
:1009E000002800F0A980099800F080F916AB43F8C0
:1009F000480D1846042100F017F991E016A80023CD
:100A000040F8343D642100F0E1F8002840F0948083
:100A10000220FFF7E9FC002800F08E80099800F022
:100A200075F916AB43F8440DE3E70220FFF7DCFC51
:100A3000002800F0818000F06FF916AB43F8400DFC
:100A4000D7E70220FFF7D0FC002875D009A91420B1
:100A500000F068F9834616A8042140F83CBD00F078
:100A6000E3F809A85946C6E7322000F07DF8B0F156
:100A7000000B61DB1BF0030F5ED1BA680BEB0603C2
:100A8000934259D80220FFF7AFFC002854D02BF036
:100A9000030BB3445E4543D0304600F0F7F816AB85
:100AA000042143F8380D184600F0BEF80436F1E78B
:100AB0004FF47A70FFF798FC00283DD0FFF7AAFCAE
:100AC00000283BD00E9B01330AD000200EA908223B
:100AD000FFF7B0FC90B30EA8FF21202200F0D6F95A
:100AE000FFF78AFC1D4801F05FFA30E016A80023EA
:100AF00040F8343D642100F069F88346E0B90220F3
:100B0000FFF772FCC0B1FFF777FC41F2883001F0CB
:100B10004BFA099800F006FAD94600F0BFF9CFE584
:100B200000F0BCF9009B1BB1002D18BF4FF000096D
:100B3000FFF762FCC4E50026094B00E0094B1B8867
:100B4000ADF8243009A8022100F06EF8B8E517B01E
:100B5000BDE8F08F702502202083B8EDA08601004B
:100B6000E23A0008E43A0008F7B500244FF47A7539
:100B70008DF807404543124B93F900305A1CE6B2FA
:100B800001D0A34210D10F4B53F8240003680DF19C
:100B900007011F6A01222B46B847012804D10A4BDE
:100BA0009DF807001E7008E00CB90124E3E74FF43C
:100BB000FA7001F0F9F94FF6FF7000B203B0F0BD22
:100BC00024240220E83A0008C0290220F8B54FF496
:100BD0007A7506464D430024104B93F900305A1C99
:100BE000E7B201D0A3420FD10D4B53F824000368A4
:100BF0003146D3F820C004222B46E047042803D115
:100C0000084B1F700020F8BD0CB90124E4E74FF435
:100C1000FA7001F0C9F94FF0FF30F8BD242402202A
:100C2000E83A0008C029022010B50A4606490346E2
:100C30000878064951F820000168CC691946A44695
:100C4000034BBDE810406047C0290220E83A000885
:100C5000A086010070B501F0D9FB094B0026187081
:100C60001C46084D23782868984208D201F0C8FB3A
:100C70002B6806440133B6F5C03F2B60F1D370BD3D
:100C8000C8290220C429022001F08ABC00F10060BA
:100C900000F5C0300068704700F1006000F5C0301A
:100CA000920001F00FBC0000054B1A68054B1B7841
:100CB0009B1A984202D2104401F0A2BB0020704758
:100CC000C4290220C829022038B5074D04462868E7
:100CD000204401F09DFB28B928682044BDE8384035
:100CE00001F0AEBB38BD00BFC4290220034610F09E
:100CF000030008D1B3F5806F06D803F10053A3F5C4
:100D0000712318687047002070470000014BC058DD
:100D1000704700BF20F4F01F014B1868704700BFF8
:100D2000002004E0F0B51F4B1F4A1B681788566867
:100D3000157AC3F30B04BC424FEA134307D09789DB
:100D4000BC4206D0178BBC4209D1022402E0002429
:100D500000E001240C2505FB04225668157AB3F542
:100D6000805F05D041F20102934208BF5A2500E09E
:100D70004125441E0C44013E0A46A2420ED216F8FA
:100D8000010F531C18B11A4603F8010CF5E72C208B
:100D9000A342107003D2931C557000E01346581AFA
:100DA000F0BD00BF002004E000240220094B5B8856
:100DB000B3F5805F05D041F20102934207D10122D1
:100DC00000E00022044B03EB8203D8787047002038
:100DD000704700BF002004E0F03A0008022802D16A
:100DE0004FF0006203E0012803D14FF40032014BC1
:100DF0009A61704700040240022802D14FF4006259
:100E000002E0012802D10222014B9A61704700BF23
:100E100000040240022804D1064A536983F40063A7
:100E200005E0012804D1034A536983F002035361AA
:100E3000704700BF0004024010B50023934203D066
:100E4000CC5CC4540133F9E710BD000030B5013863
:100E500010F8013F0C4663B12578AB4201F1010166
:100E600007D10AB1013AF3E75AB294F90030D01A27
:100E700030BD002AF8D1104630BD000002460346BE
:100E8000981A13F9011B0029FAD17047024403464E
:100E9000934202D003F8011BFAE77047024B1A781D
:100EA000024B1A70704700BFC02902202424022080
:100EB00038B5164D164C284600F0B6FB214628469C
:100EC00000F0DEFB23681348DA6ED2F8043843F0F2
:100ED0000203C2F8043801F067F820680E4900F0F8
:100EE000E1FC23680D48DA6E0D49D2F8043823F08E
:100EF0000203C2F80438A8424FF4E1330B6003D078
:100F0000BDE8384000F0EEBA38BD00BF882E0220A0
:100F1000983C000840420F002C3C0008CC290220DD
:100F2000A829022038B50C4B1A780C4B53F82240F4
:100F30000B4B9C4205460DD00A4B00211846182247
:100F4000FFF7A4FF0346056019462046BDE8384078
:100F500000F0C8BA38BD00BFC0290220E83A000836
:100F6000882E0220A8290220024A136843F0C003F9
:100F70001360704700780040044B5A6810439A6829
:100F800058600AB1181D1047704700BFCC290220D5
:100F9000F8B53E4EF56D2F68EC692C62230718D02A
:100FA00014F0080F0CBF00208020E10748BF40F07C
:100FB0002000A20748BF40F04000630748BF40F44C
:100FC0008070202383F31188FFF7D6FF002383F37B
:100FD0001188E10509D5202383F311884FF40070AF
:100FE000FFF7CAFF002383F31188A2060ED5202342
:100FF00083F3118896F86430696A2448194000F038
:101000007FFA002383F31188EC69EEE73B0619D5DC
:10101000200617D5202383F311881D4800F0D8F946
:10102000002809DA0820FFF7A7FF27F080032B60CC
:10103000002383F3118805E0A862002383F311885D
:10104000EC69E5E779060ED562060CD5202383F31B
:101050001188F26C336D9A4202D10C4B1B6C6BB948
:10106000002383F31188E30604D5B26E13690BB134
:1010700050699847BDE8F84001F016BB102027F0F2
:101080004007FFF779FF2F60EAE700BFCC29022075
:10109000042A022013B5104C204600F017FA04F180
:1010A000140000940D494FF40072002300F0DCF8A6
:1010B00004F1380000940A490A4B4FF4007200F022
:1010C00053F9094BE365094B236652200B2102B00B
:1010D000BDE8104000F058B8CC290220382A022080
:1010E000382C0220690F00080078004080F937038F
:1010F000224B002908BF1946037C8166012B30B5BD
:101100000CD11F4B984209D11E4B1A6C42F0804201
:101110001A641A6E42F080421A661B6E0B68026EE9
:10112000C46D02EB5302B2FBF3F34A68150442BFED
:1011300023F0070503F0070343EA4503E3608B68E8
:1011400043F040036360CB6843F00103A36042F4C3
:10115000967343F00103236051054FF0FF33236280
:1011600008D512F0102204D0B2F1805F02D13F23E3
:1011700000E07F2380F8643030BD00BF243B0008CE
:10118000CC2902200038024000F1604300F01F0229
:10119000400903F5614309018000C9B200F16040D4
:1011A00083F8001300F5614001239340C0F88031BB
:1011B00003607047F8B51546826806690B4695428C
:1011C000816988BF8568761AB5420446184605D2FB
:1011D0002A46FFF731FEA3692B4411E00CD93246B1
:1011E000FFF72AFEAF1B3A463044E168FFF724FEC2
:1011F000E3681F44A76104E02A46FFF71DFEE36889
:10120000A361A3685B1BA3602846F8BD83682DE932
:10121000F04104469A421546266988BF85684069B0
:10122000361AB5420F4605D22A46FFF705FE636916
:101230002B4411E00CD93246C6EB0508FFF7FCFD44
:10124000E068B9194246FFF7F7FDE368434403E05D
:101250002A46FFF7F1FDE3686361A3685B1BA360A7
:101260002846BDE8F081000010B50A440024C3619F
:10127000029B006040608460C160816141610261E5
:10128000036210BD08B582694369934204D1826844
:1012900012B14FF0FF3008BD8268013282605A1CE3
:1012A00042611970426903699A4201D3C36843617C
:1012B000002100F095FE002008BD000070B520233D
:1012C00004460E4683F31188A56845B92046314689
:1012D00000F076FE0028F7DA85F3118870BDA36868
:1012E000A269013BA360531CA36115782269934254
:1012F00024BFE368A361E3690BB12046984700234C
:1013000083F31188284670BD2DE9F0479A460546BB
:101310000E469046D0F81C90202383F31188144683
:10132000DCB1284631462246FFF744FF074630B974
:101330002846514600F044FE0028F1D00DE0B9F1F6
:10134000000F01D02846C847002383F311882023CB
:10135000E41B3E4483F31188E2E7002383F3118802
:10136000C4EB0800BDE8F0878260C3610A44009BBB
:1013700000604060C1608161416102610362704749
:10138000F8B504460E461746202383F31188A56856
:1013900045B92046394600F013FE0028F7DA85F3F8
:1013A0001188F8BDA368013BA36063695A1C6261A0
:1013B0001E70236962699A4224BFE3686361E3692E
:1013C0000BB120469847002080F31188F8BD00003B
:1013D000836942699A4210B504D1826812B14FF014
:1013E000FF3010BD8268013282605A1C82611C7815
:1013F00003699A4201D3C3688361002100F0F0FDC4
:10140000204610BD2DE9F0479A4605460E46904607
:10141000D0F81C90202383F311881446DCB12846B1
:1014200031462246FFF7F2FE074630B928465146BC
:1014300000F0C6FD0028F1D00DE0B9F1000F01D099
:101440002846C847002383F311882023E41B3E4429
:1014500083F31188E2E7002383F31188C4EB0800CB
:10146000BDE8F087026843681143016003B1184783
:1014700070470000002070471430FFF745BF0000A0
:1014800014304FF0FF33FFF73FBF00003830FFF755
:10149000B9BF000038304FF0FF33FFF7B3BF000093
:1014A0001430FFF70BBF000014304FF0FF31FFF78F
:1014B00005BF00003830FFF763BF000038304FF041
:1014C000FF32FFF75DBF0000FFF7E4BD044B036090
:1014D000002343608360C36001230374704700BF2F
:1014E0003C3B000810B52023044683F31188FFF726
:1014F000FFFD02232374002383F3118810BD000035
:1015000038B5C36904460D461BB904300421FFF702
:10151000A9FF04F114002946FFF7B4FE002806DAFB
:10152000201D4FF48061BDE83840FFF79BBF38BDF8
:10153000026843681143016003B118477047000017
:101540000020704713B5446BD4F894341A681178AE
:10155000042915D1217C022912D11979128901237C
:101560008B4013420CD101A904F14C0001F0A0FE04
:10157000D4F89434024619791868019B00F0E2F916
:1015800002B010BD143001F023BE000014304FF043
:10159000FF3301F01DBE00004C3001F0F7BE00002B
:1015A0004C304FF0FF3301F0F1BE0000143001F079
:1015B000F3BD000014304FF0FF3101F0EDBD00002D
:1015C0004C3001F0C3BE00004C304FF0FF3201F050
:1015D000BDBE0000D0F8942438B5136819780429EA
:1015E000054601D0012038BD017C0229FAD11279CB
:1015F0005C89012090400440F4D105F1140001F011
:1016000081FD02460028EDD0D5F894341868597948
:101610004FF4807300F084F9204638BD406BFFF72B
:10162000D9BF0000704700007FB5124B0360002354
:1016300043608360C3600446012502260E4B057497
:1016400029460193029004F18402009614304FF46D
:10165000807301F033FD094B01930096029404F16D
:101660004C00294604F523724FF4807301F0FCFD11
:1016700004B070BD643B00081D1600084515000845
:101680000B68202282F311880A7903EB8202106230
:101690004A790D3243F822008A7912B103EB8203B2
:1016A000186202230374C0F89414002383F3118892
:1016B0007047000038B5037F044613B190F85430EA
:1016C000ABB9201D01250221FFF732FF04F1140000
:1016D00025776FF0010100F08FFC84F8545004F17D
:1016E0004C006FF00101BDE8384000F085BC38BD0A
:1016F00010B5012104460430FFF71AFF00232377B9
:1017000084F8543010BD000038B50446002514306C
:1017100001F0ECFC04F14C00257701F0BDFD201D2B
:1017200084F854500121FFF703FF2046BDE83840FC
:10173000FFF750BF90F85C3003F06003202B19D105
:1017400090F85D20212A0AD0222A4FF000030CD005
:10175000202A0FD1084A02650722426507E0064B9E
:10176000036507234365002301E003654365836543
:10177000012070470020704725240220D0F89434BF
:1017800037B51A681178042904461AD1017C022958
:1017900017D11979128901238B40134211D100F11D
:1017A0004C05284601F03CFE58B101A9284601F03D
:1017B0007FFDD4F89434024619791868019B00F033
:1017C000C1F803B030BD000000EB8103F7B51C6A1F
:1017D00006460D465CB3202383F3118806EB85078C
:1017E000201D0821FFF7A4FEFB685B691B684C34D1
:1017F00013B1204601F06AFD204601A901F058FD11
:10180000024618B130462946019B0BE0FB685A6935
:10181000116849B11A8A531E0B4005D1304629463A
:1018200006F15C0200F08EF8002383F3118803B008
:10183000F0BD00000D3138B550F82140DCB1202357
:1018400083F31188D4F894241368527903EB82034C
:10185000DB689B695D6845B1201D0421FFF768FEC8
:1018600004F11400294601F057FC2046FFF7B2FEB0
:10187000002383F3118838BD7047000001F008B8D9
:10188000012303700023436000F1200200F13401C2
:10189000002342F8043F8A425361F9D10381438116
:1018A0007047000038B50446202383F311880025D3
:1018B0004160C560056145618561C561056200F0F3
:1018C000F7FF0223237085F3118838BD70B500EB54
:1018D000810306465069DA600D46144618B10021AE
:1018E0001022FFF7D3FAA06918B100211022FFF7E8
:1018F000CDFA30462946BDE8704001F0A5B8000099
:10190000028902F001020281428902F00102428151
:101910000022026142618261C261026201F02AB961
:10192000F0B500EB81044689E4680125A4698D4087
:101930003543458123600023A2606360BDE8F04029
:1019400001F044B9F0B500EB81040689E468012593
:1019500064698D403543058123600023A260636084
:10196000BDE8F04001F0BEB970B502230025044681
:101970000370A0F8645080F8665080F867500581C5
:101980004581C560056145618561C561056280F875
:101990004C5000F0F3FF63681B6823B120462946D2
:1019A000BDE87040184770BD436802781B6880F836
:1019B0006820052202700BB104211847704700000F
:1019C000436890F868201B6802700BB10521184726
:1019D00070470000F8B590F84C30044613B100236E
:1019E00080F84C30204604F15C0201F0E5F86368B1
:1019F0009B6833B994F85C3013F0600640F0F680D1
:101A000005E020469847002840F00281F2E794F86C
:101A10005D5003F07F0343EA052540F202339D4207
:101A200000F0D38014D8022D00F0A48004D855B360
:101A3000012D00F09880D9E0B5F5817F00F0B480E9
:101A4000B5F5407F30D0B5F5807F40F0CF8021E004
:101A500040F201639D4206D8B5F5C06F4AD2B5F594
:101A6000A06F2FD0C2E0B5F5106F58D040F60243FA
:101A70009D4278D0B5F5006F40F0B88004F167035F
:101A80002365012349E004F16403236502236365B0
:101A9000A565BDE094F85E30012B40F0A780B4F856
:101AA000643023F0020308E094F85E30012B40F02C
:101AB0009D80B4F8643043F00203A4F864302665D6
:101AC00066656FE0B4F85C30B3F5A06F0ED194F8A2
:101AD0005E3084F86630204600F0AAFF63681B6819
:101AE00013B1204601219847032323700023236567
:101AF00063653DE0626894F8617094F86030556801
:101B000094F85F1094F85E20204643EA0723A84724
:101B100000286BD0436823650368636542E023783F
:101B2000042B10D1202383F311882046FFF7E8FE11
:101B300086F31188636884F867601B68032121704D
:101B40000BB12046984794F85E30002BCED084F835
:101B500067300423237063681B68002BC6D02046BF
:101B600002219847C2E74E4B236502236365002399
:101B7000A3654DE094F8601011F0800F204601F04D
:101B80000F0102D001F00AF801E000F0F9FF01288E
:101B900005D002282AD1434B2365606502E0424B01
:101BA00023656565A66533E094F85E30F3B994F873
:101BB000603013F00F0199D01A06204602D501F0CB
:101BC00073FA93E701F066FA90E794F85E306BB928
:101BD00094F8603013F00F0188D01B06204602D520
:101BE00001F04EFA82E701F041FA7FE7204600213A
:101BF00001F046FA2046002101F038FA63681B68BC
:101C000013B1204606219847062384F84C30F8BDCE
:101C100094F8632094F8623043EA0223626D9A429A
:101C200088BF636594F95C30616D002B0D464FF001
:101C3000200317DA59B1092284F84C2083F3118864
:101C400000212046226D636DFFF77CFE16E0142212
:101C500084F84C2083F3118820460A460B46FFF790
:101C60005FFE19E071B1152284F84C2083F31188CE
:101C700000212046226D636DFFF752FE002383F39F
:101C80001188F8BD0B2284F84C2083F3118820467C
:101C90000A460B46FFF756FE85F31188F8BD00BFD4
:101CA0008C3B0008903B0008943B000838B590F846
:101CB0004C300446152B4DD8DFE803F03C4C4C4C1F
:101CC0004C4C3C4C4C0B27374C4C4C4C4C4C4C4CDF
:101CD0003C3C90F8631090F86230426D43EA012377
:101CE0009A4212D2C3681D8AB2FBF5F305FB132595
:101CF0005DB9202383F3118829462A462B46FFF736
:101D000021FE85F311880A2322E0142384F84C3045
:101D1000202383F3118800210B4620460A46FFF753
:101D2000FFFD002383F3118838BD836D03B198470D
:101D300000230DE0002101F0A3F92046002101F06D
:101D400095F963681B6813B120460621984706235E
:101D500084F84C3038BD000090F84C20152A38B576
:101D6000044631D80123934040F641621A40DAB963
:101D700013F480150FD19B0226D50B2380F84C302D
:101D8000202383F3118829462A462B46FFF7DAFDE4
:101D900085F3118838BDC3689B695B68A3B9836DFF
:101DA00003B1984700230DE0002101F069F92046B6
:101DB000002101F05BF963681B6813B1204606211E
:101DC0009847062384F84C3038BD0000024B0022AF
:101DD0001B605B609A607047382E022000230374FA
:101DE0008268054B1B6899689142FBD25A68036070
:101DF0004260106058607047382E022008B52023DA
:101E000083F31188037C032B03D0042B05D04BB93B
:101E10000EE0436900221A6004E090E80C001A60AA
:101E2000026853604FF0FF334361FFF7D7FF002391
:101E300083F3118808BD0000002303748268054BFA
:101E40001B6899689142FBD85A6803604260106031
:101E500058607047382E0220054B196908741868BD
:101E600002681A605360186101230374FEF75CBABC
:101E7000382E022030B54B1C87B005460A4C0DD0D9
:101E800023690A4A01A800F0D3F82846FFF7E4FFC7
:101E9000049B2BB101A800F007F901E0FFF7DCFF7C
:101EA0002369586907B030BD382E0220FD1D000897
:101EB00038B50C4D41612B6981689A68914204469E
:101EC00003D8BDE83840FFF789BF1846FFF786FF03
:101ED00001232C61014623742046BDE83840FEF7FB
:101EE00023BA00BF382E0220044B1A681B69906881
:101EF0009B68984294BF002001207047382E022032
:101F000010B5084C236820691A68226054600122C9
:101F100023611A74FFF790FF01462069BDE8104065
:101F2000FEF702BA382E02208260022202740022DA
:101F3000427470478368A3F17C0243F80C2C026959
:101F400043F83C2C426943F8382C074A43F81C2CD0
:101F5000C26843F8102C022203F8082C002203F870
:101F6000072CA3F1180070474103000810B5202387
:101F700083F31188FFF7DEFF00210446FFF798FF87
:101F8000002383F31188204610BD0000024B1B691B
:101F900058610F20FFF760BF382E0220202383F303
:101FA0001188FFF7F3BF000008B50146202383F333
:101FB00011880820FFF75EFF002383F3118808BD16
:101FC00049B1064B42681B6918605A601360436050
:101FD0000420FFF74FBF4FF0FF307047382E02202C
:101FE0000368834206D01A6802605060596118463F
:101FF000FFF7F4BE7047000038B504460D46206870
:10200000A04206D0036823605C604561FFF7E6FEEE
:10201000F5E738BD054B03F114025A619A614FF0A0
:10202000FF32DA6100221A62704700BF382E0220A8
:10203000F8B503614FF08043C2605C6A194B1A46E1
:10204000012998BF022152F8145F954206461F46A7
:102050000AD1586198611C62056045608160081969
:10206000BDE8F84001F0FCB9186AAB68241A0C19F5
:1020700005D29C4205D2204401F000FA01E02D680F
:10208000E41AAB68A342FAD36B68736035601E60D4
:102090006E60B460A9684FF0FF33091BA960FB6153
:1020A000F8BD00BF382E022010B51A4C234653F855
:1020B000141F81420ED0416802680A6002685160B4
:1020C0009A424FF00001C16023D0916883680B44AD
:1020D000936010BD0A68626100209A425360C86034
:1020E00003D1BDE8104001F0C3B988689368034488
:1020F00093604FF08042206A526A121A9A4208D2C4
:10210000991A012998BF931C1844BDE8104001F0AA
:10211000B5B910BD382E022000207047FEE7000040
:102120004FF0FF3070470000022906D0032906D087
:102130000129064818BF0020704705487047032A48
:102140009ABF044B03EBC20000207047A03C00087C
:10215000BC3B00082C24022070B5044608460D46FE
:10216000FEF78CFE06462046013403783BB1294633
:10217000F2B2FEF76BFE0028F5D1012070BD1846C3
:1021800070BD00002DE9F04380469BB008460C4628
:102190001646FEF773FE3B49C5B22046FFF7DCFF4B
:1021A00008B10935EDB220463749FFF7D5FF08B130
:1021B0001035EDB2632D01AF01DC3D4619E0384624
:1021C000214601F085FC3FE0B9F1250F35D12046CD
:1021D0002C490722FEF73AFE88B92C4B2A4603F118
:1021E000100153F8040B42F8040B8B42F9D1073469
:1021F000103594F80090B9F1000FE5D122E02046A7
:1022000021490822FEF722FEB8B92149AB1C11F87A
:10221000012F20484FEA121E02F00F021EF800E0C4
:10222000125C03F8012C1C4A03F802EC914203F102
:102230000203ECD118350834DBE785F8009001344F
:102240000135D6E785F800903846FEF717FEC0B294
:10225000431C5B0088E84800337003237370023628
:102260000023DAB2824206F1020607D2FA5C06F8CF
:10227000022C002206F8012C0133F2E71BB0BDE866
:10228000F08300BFE83B0008F03B0008F93B000882
:102290001FF4F01F0A3C00082BF4F01F08B52023A0
:1022A00083F311880348FFF769FA002383F3118849
:1022B00008BD00BF882E022010B50446052924D889
:1022C000DFE801F013230313131A202383F311888B
:1022D00001210E4AFFF7FAFA204602210C4AFFF7C5
:1022E000F5FA0C48FFF710FA0CE0202383F311886D
:1022F0000848FFF7DFF905E0202383F3118805483C
:10230000FFF7F6F9002383F3118810BD983B00080E
:10231000C43B0008882E022038B50C4D0C4C0D49EA
:1023200005F108002246FFF72DFF05F1100004F12A
:10233000CA020949FFF726FF05F1180004F5CA7221
:102340000649BDE83840FFF71DBF00BF2C2402201E
:10235000403302201B3C00081F3C0008F03B0008F3
:10236000BFF34F8F024BDB68DB03FBD4704700BF2A
:10237000003C024008B5074B1B7853B9FFF7F0FF4C
:10238000054B1A69002ABFBF044A5A6002F188321D
:102390005A6008BDD1350220003C02402301674548
:1023A00008B5054B1B7833B9FFF7DAFF034A136909
:1023B00043F00043136108BDD1350220003C0240C8
:1023C0000B2830B513D80B4A0B4C137863B94FF078
:1023D00000610A4D44F8231055F8235001330C2BAB
:1023E0002944F6D10123137054F8200030BD002099
:1023F00030BD00BFD0350220A0350220A83C000827
:10240000014B53F820007047A83C00080C2070478F
:102410000B2810B5044601D9002010BDFFF7D0FFEE
:10242000064B53F824100A4643189B1A22B11B6826
:102430000133F1D1043AF7E7012010BDA83C0008B0
:102440000B2838B5044635D81B4DFFF789FFFFF739
:1024500091FFF323EB60FFF783FF0C22B4FBF2F351
:1024600002FB1343DB00DBB243F4007343F00203CF
:102470002B612B6943F480332B61FFF771FF2046FA
:10248000FFF79EFF0D4B53F824300344BFF34F8FEB
:10249000984204D20A4AC2F85C022030F8E7BFF33F
:1024A0004F8FBFF36F8FFFF77BFF2046BDE83840AB
:1024B000FFF7AEBF002038BD003C0240A83C00083A
:1024C00000ED00E012F001032DE9F04707468846D1
:1024D00016465DD10244B2F1026F59D22E4B1B68F1
:1024E00013F0010354D0FFF745FF2C4BF322DA60C1
:1024F000FFF736FF032E01D8C14619E0BB07FBD119
:10250000264C236923F440732361236943F4007349
:1025100043F00103236158F8045B3D60BFF34F8F24
:10252000FFF71EFF3B68AB4223D1043E0437E1E7CF
:10253000C9EB06034344194CC8EB0705012B4D4476
:1025400023691DD923F440732361236943F4807305
:1025500043F001032361CA4639F8023B2B80BFF3E5
:102560004F8FFFF7FDFE2D88BAF80030ADB2AB42B9
:10257000DED0236923F001032361FFF711FF07E099
:1025800023F001032361FFF70BFF0120BDE8F08773
:102590000020BDE8F08700BF00380240003C024048
:1025A00010B5084C237828B153B9FFF7E3FE012397
:1025B000237010BD23B12070BDE81040FFF7F0BEBE
:1025C00010BD00BFD135022010B50244D2B29042F6
:1025D00007D0441C034B80001B5841F8043BE0B279
:1025E000F5E710BD50280040104B10B51C6F2404B7
:1025F0005FBF1C6F44F400741C671C6F5CBF44F425
:1026000000441C670A4C2368024443F4807323602F
:10261000D2B2904208D0074B441C8000034451F8CA
:10262000040B1860E0B2F4E710BD00BF00380240B0
:10263000007000405028004007B5002001A9012289
:10264000FFF7C2FF019803B05DF804FB07B502A9CC
:10265000012241F8040D0020FFF7C6FF03B05DF82A
:1026600004FB0000034B1B689B0042BF024B01228E
:102670001A70704774380240D2350220014B187826
:10268000704700BFD2350220064A536823F0010389
:102690005360EFF30983683383F30988002383F3DE
:1026A0001188704730EF00E010B5202383F31188C4
:1026B000104B5B6813F4006318D0F1EE103AEFF39F
:1026C00009844FF0807344F84C3C0B4BDB6844F8B2
:1026D000083CA4F1680383F30988FFF705FC08B1FF
:1026E000064B00E0064B44F8503C10BD83F31188C4
:1026F00010BD00BF00ED00E030EF00E05103000826
:102700005403000830B5BFF34F8FBFF36F8F1A4BE0
:102710000021C3F85012BFF34F8FBFF36F8F5A6978
:1027200042F400325A61BFF34F8FBFF36F8FC3F88B
:102730008410BFF34F8FD3F88020C2F34E33C2F31F
:10274000C902590143F6E0740C4011460A4844EAB4
:10275000817511F1FF31C0F86052F7D213F1FF33E8
:10276000EFD2BFF34F8F436943F480334361BFF32C
:102770004F8FBFF36F8F30BD00ED00E0FEE700002C
:10278000084A094B09498B4204D252F8041F43F806
:10279000041BF7E7064A934203D2002243F8042BB6
:1027A000F8E77047A83E0008E0380220E038022031
:1027B000E0380220036F30B5C46E9D68002204EB40
:1027C0004213013200214FF0FF30AA42C3F8001932
:1027D000C3F81019C3F80809C3F8001BC3F8101B8D
:1027E000C3F8080BEBD94FF00113C4F81C3830BD07
:1027F000890141F02001016103699B06FCD412208C
:1028000000F0CCBE2DE9F043204D05EB8003D5F858
:102810006C90D3F80CC0DCF8142000F1010ED2F853
:10282000008009EB0E3E516841450CD3E96E01234F
:10283000D1F8342803FA00F022EA0002C1F8342863
:102840001846BDE8F083BCF81040C1EB0803A34272
:1028500028BF234609EB4014D4F81849A4B2B3EBBF
:10286000840F0FD8946826463768CEF800709F1BF7
:102870002744042F01D90436F6E71C440B44946026
:102880005360D0E70020BDE8F08300BFD4350220BC
:1028900010B5054C2046FEF7F3FF4FF0A043E3666A
:1028A000024B236710BD00BFD4350220D83C00087E
:1028B0000378012B70B50546C46E51D1294B98425F
:1028C0001BD1294B5A6B42F080025A635A6D42F079
:1028D00080025A655A6D5A6942F080025A615A69FB
:1028E00022F080025A6143200E215B69FEF74CFC06
:1028F0001E4BE3601E4BC4F800380023C4F8003EB2
:10290000C0232360EE6E4FF40413A3633369002BDE
:10291000FCDA012333610C2000F040FE3369DB0751
:10292000FCD4122000F03AFE3369002BFCDA0026BA
:10293000A6602846FFF73EFF6B68C4F81068DB68A6
:10294000C4F81468C4F81C680BB90A4B00E00A4BC1
:10295000A3614FF0FF336361A36843F00103A360F9
:1029600070BD00BFD4350220003802404014004042
:1029700003002002003C30C0083C30C070B5C46E7B
:10298000054600212046FFF733FF296F00234FF053
:1029900001128E68C4F83438C4F81C2804EB4312C2
:1029A0004FF000600133C2F80009B342C2F8000BD7
:1029B0004FF0FF30C2F80809C2F8080BEED90B68D7
:1029C0006B67EA6E0B68636210231361136913F07F
:1029D0001006FBD1122000F0E1FDD4F8003823F4FA
:1029E000FE63C4F80038A36943F4402343F01003A6
:1029F000A3610923C4F81038C4F814380A4BEB60FB
:102A00004FF0C043C4F8103B084BC4F8003BC4F877
:102A10001069C4F800396B6F03F1100243F480139E
:102A20006A67A36270BD00BFE43C000840800010EC
:102A3000C26E90F86610D2F8003823F4FE6343EAC1
:102A40000113C2F8003870472DE9F0410FB200EBD6
:102A500087080D46D8F80C10C46E0E6806F0030304
:102A6000022B07D0032B07D03D4A3E4E012B18BF47
:102A7000164602E03C4E00E03C4E6A01A3184FF0BF
:102A8000000EC3F810EB8B6905F1100C8BB1B1F897
:102A900012E005F158035B0146EA0E0E44F803E02C
:102AA0004FF0010ED4F81C380EFA0CFE4EEA030368
:102AB0000FE004EB471EDEF8003B23F40043CEF8A2
:102AC000003BD4F81C384FF0010E0EFA0CFE23EA3E
:102AD0000E032244C4F81C380023C2F810394B6995
:102AE00005F13F020BB30B8A898B9B08012988BF34
:102AF0004B43416F04EB82025F1841EA034347678F
:102B0000294653602046FFF773FED8F80C301B8A25
:102B100043EA85531E4305F148035B01E650012358
:102B2000D4F81C28AB40134315E004EB8202104B91
:102B3000536020462946FFF75BFE04EB4713D3F8AA
:102B4000002922F40042C3F80029D4F81C280123EC
:102B5000AB4022EA0303C4F81C38BDE8F08100BF93
:102B600000800010008004100080081000800C100D
:102B700000040002026F12684267FFF71BBE0000EC
:102B80005831C36E49015B5813F4004004D013F46C
:102B9000001F14BF01200220704700004831C36E9F
:102BA00049015B5813F4004004D013F4001F14BF14
:102BB000012002207047000000EB8101CB68196AF8
:102BC0000B6813604B6853607047000000EB810393
:102BD00030B5DD68AA691368D36019B9402B84BF8A
:102BE0004023136014686B8AC26E013C1C44B4FB22
:102BF000F3F46343E004033340F0C04023F00303E5
:102C0000034302EB411009B2C0F8103B2B6803F0FC
:102C10000303012B0ED1D2F8083802EB411013F454
:102C2000807FD0F8003B14BF43F0805343F0005343
:102C3000C0F8003B02EB4112D2F8003B43F00443E2
:102C4000C2F8003B30BD00002DE9F041244DEE6E8E
:102C500006EB40130446D3F8087BC3F8087B38071B
:102C60000AD5D6F81438190706D505EB840328468B
:102C7000DB6821465B689847FA072ED5D6F81438EA
:102C8000DB072AD505EB8403D9688B69C4B94A8A66
:102C90005E68B6FBF2F002FB10628AB91868DA6867
:102CA00090420DD2121A83E81400202383F3118876
:102CB0000B482146FFF78AFF84F31188BDE8F081B5
:102CC0006A890123A34022EA03036B81CB6823B105
:102CD00021460348BDE8F0411847BDE8F08100BF38
:102CE000D435022000EB8103F0B5DD68C36E6A695C
:102CF0001668D6604C011EB91C444FF400220FE048
:102D000019B9402E84BF4020106012682F8A42F00B
:102D10000056013AD0191C44B0FBF7F246EAC24211
:102D2000C4F810292A6802F00302012A0AB20ED15F
:102D3000D3F8080803EB421410F4807FD4F800099C
:102D400014BF40F0805040F00050C4F8000903EB7D
:102D50004212D2F8000940F00440C2F80009D3F84A
:102D6000340801228A400243C3F83428F0BD000031
:102D7000F8B504461D48C56E05EB4413D3F8086941
:102D8000C3F80869F10722D5D5F81038DA071ED53F
:102D900000EB8403D9684B691F68DA6897420CD24C
:102DA000D21B00271A605F60202383F3118821461D
:102DB000FFF798FF87F3118809E002890123A340F8
:102DC00022EA030303818B680BB12146984733063F
:102DD0000AD5D5F834280123A340134204D0204655
:102DE000BDE8F840FFF70EBDF8BD00BFD4350220A6
:102DF0009D482DE9F843C46E6369A5691D4015F42B
:102E0000805F6561064602D0FEF7AEFD27E1002D2A
:102E100012DAD4F8003E94489B071EBFD4F8003E57
:102E200023F00303C4F8003ED4F8043823F0010370
:102E3000C4F80438FEF7C4FD2F0502D58A48FEF712
:102E4000B3FDA8040CD5D4F8083813F0060FE368D6
:102E500023F470530CBF43F4105343F4A053E360C6
:102E6000290704D57368DB680BB17F489847EA02ED
:102E700002D4AB0243D538E0D6F86C904FF000088E
:102E8000336F9B685FFA88F79F42F2D809EB4713CC
:102E9000D3F8002902F44022B2F5802F22D1D3F8D2
:102EA0000029002A1EDAD3F8002942F09042C3F824
:102EB0000029D3F80029002AFBDBF06E3946FFF722
:102EC00097FC32890123BB4022EA0303338106EBDE
:102ED0008703DB689B6813B16348394698473846D7
:102EE000FFF790FC08F10108CAE7F76E4FF0000801
:102EF000336F5D489B685FFA88F1994202D9EF060B
:102F00006BD51BE007EB4112D2F8003B03F44023E2
:102F1000B3F5802F0FD1D2F8003B002B0BDA42899A
:102F200001238B4022EA0303438100EB8103DB682A
:102F3000DB6803B1984708F10108D9E7F06E4A4B06
:102F4000026AC2F30A1702F00F0102F4F012B2F59E
:102F5000802F18D0B2F5402F3FD103EB8103DB68FF
:102F6000196A00231A46BB4237D09E0704BF00F5FA
:102F700080521268072B98BF0A7003F101039CBFAF
:102F8000120A0131EFE78A1C03EB82035B6899693F
:102F90000B68D1F808C04968C1EB030E002319463D
:102FA000BB4210D013F0030F04BF00F58051096835
:102FB000734538BF8CF8001003F101033CBF090AC8
:102FC0000CF1010CECE706EB8206726892699168DD
:102FD0001944916051680B4453602B03D4F818488E
:102FE0001DD5E70302D50020FFF72EFEA60302D56C
:102FF0000120FFF729FE600302D50220FFF724FE1F
:10300000210302D50320FFF71FFEE20202D50420B0
:10301000FFF71AFEA30202D50520FFF715FE6F0386
:103020001DD5E60702D50020FFF7A2FEA50702D5B1
:103030000120FFF79DFE600702D50220FFF798FEF2
:10304000210702D50320FFF793FEE20602D50420F4
:10305000FFF78EFEA30602D50520FFF789FEBDE827
:10306000F843FFF721BB00BFD4350220C36E03EB4A
:103070004111D1F8003B43F40013C1F8003B704705
:10308000C36E03EB4111D1F8003943F40013C1F8CA
:1030900000397047C36E03EB4111D1F8003B23F4B4
:1030A0000013C1F8003B7047C36E03EB4111D1F828
:1030B000003923F40013C1F80039704730B5039C80
:1030C0000172043304FB0325C361049B03630021E5
:1030D000059B00604060C1604261026185610462DD
:1030E00042628162C162436330BD00000022416AD6
:1030F00041610161C2608262C2626FF00101FEF74C
:103100007BBF000003694269934203D1C2680AB1E0
:1031100000207047181D704710B504692160C2680F
:10312000C3690132C260826923449342036124BFB0
:10313000436A03610021BDE81040FEF751BF000063
:1031400038B504460D46E36843B9237A73B920467F
:103150002946FEF735FF0028F5DA09E063691A1DF4
:103160001B68A2621344E362002038BD6FF00100C7
:1031700038BD0000C3684269013BC360C3691344A2
:1031800082694361934224BF436A4361002383629F
:10319000036B03B11847704738B50546202383F306
:1031A0001188846A2CB9FFF7CBFF10B184F3118822
:1031B00038BDAB6AEA6A13F8014BAB62934202D3A3
:1031C0002846FFF7D7FF002383F31188204638BD38
:1031D0002DE9F8431F46044688461646202383F30C
:1031E00011884FF00009A56A3DB920463946FFF71E
:1031F000A7FF10B185F3118833E0A16AE56AC9EB36
:1032000006036D1A9D4228BF1D46402D10D9434626
:1032100001F1400251F8040B43F8040B9142F9D13B
:10322000A36A403308F14008A36209F1400908E0AD
:1032300040462A46FDF700FEA36A2B44A844A36239
:10324000A944A26AE36A9A4202D32046FFF792FF9A
:10325000002383F31188B14503D2202383F311881F
:10326000C1E74846BDE8F88310B5029C01720433FB
:1032700003FB0421C36100238362C362039B0363D6
:10328000049B00604060C46042610261816104622D
:103290004262436310BD0000026AC260426A42613A
:1032A000026100228262C2626FF00101FEF7A4BED9
:1032B000436902699A4203D1C2680AB1002070478B
:1032C000184650F8043B0B6070470000C368426921
:1032D0000133C360C369134482694361934224BFCD
:1032E000436A43610021FEF77BBE000038B5044607
:1032F0000D46E36843B9237A73B920462946FEF7A1
:103300005FFE0028F5DA09E02269131DA362E36974
:103310001344E362002038BD6FF0010038BD0000A7
:1033200010B504692160C268C369013AC26082694C
:1033300023449342036124BF436A036100238362F1
:10334000036B13B1BDE81040184710BD70B52023C2
:1033500004460E4683F31188856A35B91146FFF796
:10336000C5FF10B185F3118870BDA36A1E70A36AF2
:10337000E26A01339342A36204D3E169204604392F
:10338000FFF7CEFF002080F3118870BD2DE9F843D0
:10339000994604460D469046202383F31188002762
:1033A000A66A3EB920464946FFF7A0FF10B186F352
:1033B000118831E0A06AE66AC7EB0803361A9E421C
:1033C00028BF1E46402E0CD905F1400355F8042BAA
:1033D00040F8042B9D42F9D1A36A4033A3624037E1
:1033E00008E029463246FDF727FDA36A33443544F9
:1033F000A3623744A26AE36A9A4204D3E169204691
:103400000439FFF78DFF002383F31188474503D26A
:10341000202383F31188C3E73846BDE8F883000012
:10342000026943699A4203D1C3680BB1836A0BB93D
:1034300000207047043B9B1AFAD01360C368013B1D
:10344000C360C3691A44836902619A4224BF436A14
:1034500003610023836201207047000000F044B93B
:103460004FF08043002258631A610222DA607047ED
:103470004FF080430022DA60704700004FF0804335
:1034800058637047FEE7000010B5194CFEF79EFC2C
:10349000FEF7C0FD204617498022FEF745FD0123B7
:1034A00044F8180C0374144B144AD96821F4E061F1
:1034B0000904090C0A431249DA60CA6842F08072B2
:1034C000CA60104A1049C2F8B01F116841F00101EA
:1034D00011601022DA77202283F82220002383F360
:1034E000118862B60948BDE81040FEF73FBD00BF35
:1034F000602E0220203D000800ED00E00003FA05E8
:10350000F0ED00E0001000E055CEACC5083D00082D
:103510002DE9F843204D6C69A2681F494FF08043A4
:1035200001F11408586A2B6AC61A96421ED3A26883
:103530002B6AD4F80C901344B61A22682B624245C9
:103540004FF00003C2F804801F466A61E36001D1B6
:10355000FFF78EFF87F311882069C847202383F384
:1035600011886C69A368B342E1D9D5E74A6942453D
:103570000FD033440B6291688E1B9660A2681B1AB1
:103580001344012B98BF02231844BDE8F843FFF70A
:1035900075BFBDE8F88300BF382E0220034B596881
:1035A0005A68521A8242FBD3704700BF001000E0F5
:1035B0004B6843608B688360CB68C3600B69436171
:1035C0004B6903628B6943620B68036070470000BC
:1035D000274B2848196940F2FF72114310B5196151
:1035E0001969254C21F4FF6121F00701196119695E
:1035F000196B11431963196D0A431A6521461B6D36
:10360000FFF7D6FF04F11C011C48FFF7D1FF04F1BE
:1036100038011B48FFF7CCFF04F154011948FFF7AC
:10362000C7FF04F170011848FFF7C2FF04F18C01D5
:103630001648FFF7BDFF04F1A8011548FFF7B8FFD2
:1036400004F1C4011348FFF7B3FF04F1E00112488D
:10365000FFF7AEFF04F1FC011048FFF7A9FF04F5E6
:103660008C710F48FFF7A4FFBDE8104000F09EB832
:1036700000380240000002402C3D000800040240D7
:1036800000080240000C02400010024000140240FA
:1036900000180240001C02400020024000240240AA
:1036A0000028024008B500F0F5F9FFF7EDFEFEF73F
:1036B000D9FFBDE80840FEF72FBE000070470000AC
:1036C0004FF0804310B51A69920708D500241C6199
:1036D000202383F31188FFF71BFF84F31188BDE8D3
:1036E0001040FEF7E1BF0000104B1A6C42F00102DF
:1036F0001A641A6E42F001021A660D4A1B6E936834
:1037000043F0010393604FF080436B229A624FF0C5
:10371000FF32DA6200229A615A63DA605A6001224B
:103720005A611C201A600821FDF72EBD00380240A6
:10373000002004E01B4B1A696FEA42526FEA5252B2
:103740001A611A69C2F30A021A614FF0FF301A694E
:103750005A69586100215A6959615A691A6A62F0B6
:1037600080521A621A6A02F080521A621A6A5A6AFF
:1037700058625A6A59625A6A0B4A106840F480705B
:103780001060186F00F44070B0F5007F1EBF4FF45A
:10379000803018671967536823F40073536000F092
:1037A00059B900BF0038024000700040354B364A1E
:1037B0001A64364A4FF4404111601A6842F001021F
:1037C0001A6019682F4A8907FBD5936823F0030311
:1037D00093602C4B9A6812F00C02FAD1196801F030
:1037E000F90119609A601A6842F480321A60196807
:1037F000244A8803FBD5536F43F001035367214BE1
:103800005A6F9107FBD5224A5A601A6842F08072BB
:103810001A601E4B5A685204FBD51A6842F4803273
:103820001A605968194AC803FBD5136843F400337A
:103830001360164B5B689903FBD5124B1A68920113
:10384000FBD5144A9A6040F20112C3F88C20002282
:10385000C3F89020104A40F2073111609A6842F094
:1038600002029A60074B9A6802F00C02082AF9D10A
:103870005A6C42F480425A645A6E42F480425A664C
:103880005B6E70470038024000040010007000407A
:10389000186C400900948838003C0240084A08B57A
:1038A000516913680B4003F00103536123B1054ACA
:1038B00013680BB150689847BDE80840FEF7F4BEA6
:1038C000003C014060380220084A08B5516913687D
:1038D0000B4003F00203536123B1054A93680BB117
:1038E000D0689847BDE80840FEF7DEBE003C0140C6
:1038F00060380220084A08B5516913680B4003F08C
:103900000403536123B1054A13690BB15069984709
:10391000BDE80840FEF7C8BE003C01406038022008
:10392000084A08B5516913680B4003F00803536156
:1039300023B1054A93690BB1D0699847BDE80840A7
:10394000FEF7B2BE003C014060380220084A08B5CC
:10395000516913680B4003F01003536123B1054A0A
:10396000136A0BB1506A9847BDE80840FEF79CBE49
:10397000003C014060380220174B10B55A691C68A2
:10398000144004F478725A61A30604D5134A936A6A
:103990000BB1D06A9847600604D5104A136B0BB17F
:1039A000506B9847210604D50C4A936B0BB1D06B32
:1039B0009847E20504D5094A136C0BB1506C98473F
:1039C000A30504D5054A936C0BB1D06C9847BDE8AC
:1039D0001040FEF769BE00BF003C01406038022085
:1039E0001A4B10B55A691C68144004F47C425A61A1
:1039F000620504D5164A136D0BB1506D9847230527
:103A000004D5134A936D0BB1D06D9847E00404D5EB
:103A10000F4A136E0BB1506E9847A10404D50C4A9F
:103A2000936E0BB1D06E9847620404D5084A136FA9
:103A30000BB1506F9847230404D5054A936F0BB11F
:103A4000D06F9847BDE81040FEF72EBE003C014005
:103A500060380220062008B50146FDF795FB0720D7
:103A60000621FDF791FB08200621FDF78DFB0920BB
:103A70000621FDF789FB0A200621FDF785FB1720AB
:103A80000621FDF781FB28200621BDE80840FDF74F
:103A90007BBB000008B5FFF74DFE00F00DF8FDF709
:103AA00013FDFDF7EBFEFDF7BDFDFFF707FEBDE8DB
:103AB0000840FFF7D3BC00000023044A00219950BE
:103AC0001A440833802B5160F7D1704760380220C8
:103AD000034611F8012B03F8012B002AF9D1704796
:103AE0001210121312110000882E0220CC2902207D
:103AF0000010410001105A0053544D3332463F3FED
:103B00003F3F3F3F0053544D333246375B347C35A3
:103B10005D780053544D333246375B367C375D78E1
:103B200000000000009600000000000000000000FF
:103B30000000000000000000000000000000000085
:103B40009514000881140008BD140008A914000889
:103B5000B5140008A11400088D1400087914000899
:103B60007514000800000000A11500088D1500085C
:103B7000C9150008B5150008C1150008AD150008E5
:103B8000991500088515000841150008000000007F
:103B90000000000001000000020000000000000022
:103BA000C9170008351800084000400020330220E3
:103BB000303302200200000000000000430000003B
:103BC0003C3C0008030000000000000079180008D9
:103BD0000000000010000000782E0220000000000D
:103BE000010000000000000025424F415244250022
:103BF0002553455249414C25006D526F436F6E74F9
:103C0000726F6C5A65726F4637003031323334351B
:103C100036373839414243444546006D526F0025DE
:103C2000424F415244252D424C000000B922000869
:103C300029210008351700089D22000809024300C9
:103C4000020100C032090400000102020100052443
:103C500000100105240100010424020205240600CD
:103C600001070582030800FF09040100020A0000A1
:103C70000007050102400000070581024000000026
:103C800012011001020000408304405700020102AB
:103C90000301000004030904D435022001010200DD
:103CA00012000000803C000800800000008000003E
:103CB00000800000008000000000020000000400FE
:103CC00000000400000004000000040000000400E4
:103CD000000004000000040080000000400100001B
:103CE0000500000000000000D5190008AD1C000808
:103CF000591D0008400040004C3602204C3602207E
:103D0000010000005C360220253D000868360220D4
:103D10006038022001000000853400080000000027
:103D20006D61696E0069646C650000000000802AA6
:103D300000000000AAAAAAAA00000000FFFF0000DD
:103D40000000000000A00A00440040000000000045
:103D5000AAAAAAAA00000000FFFF000000000000BD
:103D6000000000000000000000000000AAAAAAAAAB
:103D700000000000FFFF0000000000000000000045
:103D80000000000000000000AAAAAAAA000000008B
:103D9000FFFF0000000000000000000000800200A3
:103DA00000000000AAAAAAAA00400100FFFF00002C
:103DB000000000800800000000000000000000007B
:103DC000AAAAAAAA00000000FFFF0000000000004D
:103DD000000000000000000000000000AAAAAAAA3B
:103DE00000000000FFFF00000000000000000000D5
:103DF0000000000000000000AAAAAAAA000000001B
:103E0000FFFF0000000000000000000000000000B4
:103E100000000000AAAAAAAA00000000FFFF0000FC
:103E20000000000000000000000000000000000092
:103E30000000000000000000000000000000000082
:103E40000000000000000000000000000000000072
:103E50000000000000000000000000000000000062
:103E600000000000F83A00083F000000490400008C
:103E7000053B00083F00000051040000133B000810
:103E80003F000000FF009600000000080400000052
:103E9000943C00080000000000000000000000004A
:0C3EA00000000000000000000000000016
:00000001FF
